:030000000219FDE5
:03000B000200A848
:03002B000201636C
:03005B000202EDB1
:030073000202D3B3
:1000800002030406080C10182030406080040608A3
:100090000C10182030406080A0C000070F1F3F05E3
:1000A000050D050305030302C2AFC0D0C0E0206206
:1000B00017E5256002E473E525F4F58A758B00D217
:1000C00062D0E0D0D0D2AF3285268AC262E526F473
:1000D0006035306803207210758B00D0E0D0D0D22C
:1000E00095D293D297D2AF32D295D293D297206E37
:1000F0000C2066097406D5E0FDE57E4290758B0004
:10010000D0E0D0D0D2AF32758A00C28DD26201FD6C
:1001100001B7306805206602C29501B73068052036
:100120006602C29701B7306805206602C29301B724
:10013000C29430680A2066077406D5E0FDC29501B6
:10014000B7C29630680A2066077406D5E0FDC297EC
:1001500001B7C29230680A2066077406D5E0FDC276
:100160009301B7C2AFC2AD53E6EFC0D0C0E0D2D367
:10017000D2AFC2CEE52A6007207449152A21C4787F
:1001800000790020742EE580307E01F430E502789D
:10019000FF53DACF207E0343DA20307E0343DA10A8
:1001A000C2D8C271E580307E01F430E50279FFC328
:1001B000E89970CB306103752A18207403752A18EA
:1001C000885FD27020740DE52B6004152B21D44379
:1001D000DA01C2D82070024136A85F206102C270E5
:1001E000207431C3E894F0400374F0F8E8C4540F6D
:1001F00028F87984B703024114C313C3138721205D
:100200000802C313200A06C3C898F8411428F850FE
:100210000374FFF8C3E895685003E568F88822E5A1
:100220002D54066011E533C313C31324062522F5AC
:100230002250037522FF852224A824C3E524956457
:100240004002A8648825E5697002417AC3E8AA697A
:100250009A5003E8FAE4F9EAC333FBE56BF45B294F
:10026000400D256AF8E56A6002156A400B417A0A7A
:10027000C3E56A9A5002056A78FF8826C26EC3E514
:100280002694F84002D26EC3E52594404002D26421
:1002900020CF0AD0E0D0D043E610D2AD32C2CF0595
:1002A0003A7801E52A6005307402152AC3E55F94A7
:1002B00001400575620041C9756300756C00E56217
:1002C0002401F56250037562FFD0E0D0D043E61000
:1002D000D2AD32C2AFC0D053E67FC2607591008507
:1002E0005694855795759104D0D0D2AF32C2AF5392
:1002F000E6EFC2ADC0D0C0E0C0F0D2D3D2AFA8FB11
:10030000A9FCC2D8307102615453DACF207E034376
:10031000DA10307E0343DA20D271E580307E01F4BA
:1003200020E502612B88278928A17B53DACF207E24
:100330000343DA20307E0343DA10C2D8C27130742E
:1003400002A1677800E580307E01F430E502A16704
:10035000885FA14F53DACF207E0343DA20307E033B
:1003600043DA10C271206102812D53DACF207E035F
:1003700043DA10307E0343DA20C2D8D271885A891A
:100380005BC3E89558F8E99559F97B007E087A0037
:10039000C3E8948CE994005005755E00811F8821A4
:1003A00078A2E6A8216055C3E894C8E994005008F3
:1003B000E4D2E4FB7A0A61FAC3E89468E994015054
:1003C00008E4D2E3FB7A0F61FAC3E894D0E994021F
:1003D0005008E4D2E2FB7A1E61FAC3E894A0E994E3
:1003E000055008E4D2E1FB7A3C61FAC3E89498E94D
:1003F00094085008E4D2E0FB7A787E00C3E8955C6C
:10040000FCE9955DFD30E70AECF42401FCEDF434E1
:1004100000FD755E00C3EC9AED9E5003755E018889
:100420005C895D855A58855B597802A14FC3E89570
:1004300027F8E99528F9307C02A133307B02A133FB
:10044000307A02A12C2075028150E9FDE8FC816F11
:10045000E9C313F9E813F8307902A12CE9C313F9C1
:10046000E813F8307802A12CE9C313FDE813FC204F
:0E0470006126C3EC941CED940240028186EDDF
:10047E007018C3EC94C850120529C3E529940A508C
:10048E0002A167755F00D270A167E5296002152988
:10049E007888E6F97400207F087896B90302789E72
:1004AE00E624FAFEE43400FFC3EC9EFCED9FFD92C1
:1004BE0008B90310A2085007207609D27681D230EF
:1004CE007602C276A2085016B9030DECF42401FC94
:1004DE00EDF43400FD0204EC78007900A133B90389
:1004EE0015EC33FCED33FDC3EC940AFCED9400FDEA
:1004FE0050047C007D00C3EC94FFED940040067820
:10050E00FF7900A133EC8575F0A4C5F0A2F733F89E
:10051E007900400302054F78FF790002054FE9C3C9
:10052E0013F9E813F8307C0EE9600278FFC3E81384
:10053E0038F8E43400F9C3E894FFE99400400278F7
:10054E00FF885FD270206102A167741FF4552F4B94
:10055E00F52FC274EB7002D274752A1830740375BD
:10056E002A0A306102A17B20740353DAFE20740341
:10057E00752B06D0F0D0E0D0D0D2AD43E610327954
:10058E00010205AB79030205AB790A0205AB791EB0
:10059E000205AB79640205AB79C80205AB7817E4A6
:1005AE00D5E0FDD8FAD9F6227A147B780205D27AF4
:1005BE00107B8C0205D27A0D7BB40205D27A0B7BAE
:1005CE00C80205D27902B27DE4C296D5E0FDC2978B
:1005DE00D5E0FDD297D5E0FDD296D5E0FDC295E5EA
:1005EE0076D5E0FDD2957496D5E0FDD9D9EAF8D549
:1005FE00E0FDD8FBDBCEC29622C37C007D0075F0F9
:10060E000005F0EA33FAEB33FB50F6EB13FBEA137B
:10061E00FAC3E9FFE8FEE89AF8E99BF95004EFF90E
:10062E00EEF8B3EC33FCED33FDD5F0DFEDF9ECF87D
:10063E0022E889F08A20D2D4F8A9F07B0030F70B9B
:10064E007BFFF42401F8E9F43400F9E88520F0A4E6
:10065E00ADF0F8E98520F0A4AFF0FEED2EF97400B0
:10066E003FFA7C04C3EA13FAE913F9E813F8DCF451
:10067E008BF030F70AE8F42401F8E9F43400F9E8D5
:10068E0089F0C2D4F8A9F02222C3E54113F9E5405E
:10069E0013F8C3E54598F8E54699F9500CC3E8946C
:1006AE0080E994FF40160206CEC3E8947FE99400D9
:1006BE0050030206CE787F79000206CE788079FF4D
:1006CE00884A894B22E54A2547F8E54B3548F98596
:1006DE004B20E4300701F43549FA30E709C3EA94B8
:1006EE00F0401502070CC3EA940F500302070C7872
:1006FE00FF79FF7A0F02070C780079007AF0C3E5D4
:10070E00249564500AC374019524500B02072AE500
:10071E004B20E70E02072AE54B30E706884789484B
:10072E008A492278A4E6FAC3E54A33F8E54B33F951
:10073E00D13FE930E70BC3E89480E994FF4013E121
:10074E0064C3E8947FE994005002E164787F7900F5
:10075E00E164788079FFE820E715C3E52398F84037
:10076E0009C3E89401400302078B780102078BE866
:10077E00F424012523F8400302078B78FF884C22CE
:10078E0078A5E6FAA848A949D13FE930E70CC3E8B5
:10079E009401E994FF40160207BFC3E894FFE99461
:1007AE000050030207BF78FF79000207BF78017976
:1007BE00FFE920E715C3E54C98F84009C3E894011A
:1007CE0040030207E678010207E6E8F42401254C0F
:1007DE00F840030207E678FF88242278FFC26420DF
:1007EE00693D206A12D264C3E541940A4009C3E50B
:1007FE002594405002C26479A1E76023E541601F51
:10080E0074FF8541F0848539F0306A0375F005A4D4
:10081E00F8C5F0600278FFC3E895675002A86788B4
:10082E006622C3E5409440E5419401E56650031409
:10083E000141046002F566220208492275E8902201
:10084E007883E6FFE5E820ECF7A8BDA9BE0573C3E3
:10085E00E57394084052757300E9FA79A0E7604495
:0E086E00EA7007E574601B020884C3E8957405
:10087C006010E5745006600C140208900460F902D4
:10088C000890E574F574C3946D401B7564C0C394F3
:10089C00044013756480C39404400B756440C39486
:1008AC0004400375640075BB0822E564F46002051E
:1008BC0064E573B4070375BB1022743279A687F014
:1008CC00A4C5F0A2F733F8C3E895644002A8648885
:1008DC00228824882588268867227540007541F077
:1008EC0022C2AF75C820A8CCA9CDAA3A30CF010A34
:1008FC0075C824D2AFAB3BAC3C883B893CC3E89B6E
:10090C00F8E99C206908F93067024102215FAD3D8E
:10091C008A3DF9EA9DFA600478FF79FFAE3EAF3F5D
:10092C008B3E8C3FC3EC9FFCC3E99CF542A83BA9D2
:10093C003CC3E89EF8E99FF9C3E54113FBE540137E
:10094C00FAE82AF540E93BF54150067540FF754140
:10095C00FF21A9AA40AB41AC40AD417E047F02C34C
:10096C00EB940440021E1FC3EB940840021E1FC3ED
:10097C00ED13FDEC13FCDEF7C3EA9CFAEB9DFBEFE9
:10098C006009C3E913F9E813F8DFF7EA28FAEB3941
:10099C00FB8A408B4150067BFF8B408B41C3EB9411
:1009AC00025002D2673069047F0321D47892E6FFAB
:1009BC00C3E537948240110FC3E53794A040010F73
:1009CC00C3EF940640027F057E05E541C4540FF940
:1009DC00E541C454F0F8E540C4540F28F8C3E89E30
:1009EC00FAE99400FB4009C3EA9402EB940050042A
:1009FC007A02E4FB414EAA40AB41EBC4FEEAC4547C
:100A0C000F4EFCC3EA9CFAEB9400FBC3E813C31330
:100A1C00F8EA28FAEB3400FB8A408B41C3EB9402D2
:100A2C004002C2677805EBC4FE7B00EAC4540F4E4B
:100A3C00FAC3EA98FA4005C3940250027A027892FB
:100A4C00E6FF306002414E855256855357D26043C3
:100A5C00E680C3E49AF8E49BF930670241E8E8FACF
:100A6C00E9FBD3E913FDE813FC88528953C3EF94D7
:100A7C00036038EF20E00DE82CF8E93DF9ECFAEDD5
:100A8C00FB020AA3E828F8E939F9C3E82402F8E9DB
:100A9C003400F97AFE7BFFC3EF9403400E8A548B2B
:100AAC0055884E894F8C508D51611C885489558ABC
:100ABC004E8B4F8C508D51306920C3E533940340DD
:100ACC0019E542A2E713F8E555F4240138400B2050
:100ADC00E7087554FFF42401F555611CE8FAD3E8D6
:100AEC0013FC8852C3EF94036020EF20E007E82C3E
:100AFC00F8ECFA6108E8282402F87AFEC3EF9403B4
:100B0C0040088A54884E8C50611C88548A4E8C50F4
:100B1C00E56BC3335002646BF56B30600261267574
:100B2C003402D26043E680E52D54066026A840A925
:100B3C0041C3E913F9E813F8C2AF53E67F7591008E
:100B4C00C3E498F594E499F595759104D26043E665
:100B5C0080D2AF22D265754400752000306B0375CE
:100B6C002040020B7FD265754400752040306B032A
:100B7C00752000D2AF7801206722E52D5406600263
:100B8C00C265C3E54194054013780294054008788A
:100B9C0003940540027806306902780A206019E552
:100BAC0044601530690AC3E53394034003D5340619
:100BBC00D2AFD26C8150712ED2AF0000C2AF206781
:100BCC0026E541C3FB940F40027B0FEB24053073E9
:100BDC000123306A02742820620123F930690279FA
:100BEC0082E58BC39940B50544E59B5440B5200282
:100BFC00813A30690A08C3E8940A40010861A820C8
:100C0C006502617FC26553E67F7591003067107590
:100C1C0094007595FE759104D26043E680617FAEB9
:100C2C0040AF41C3E49EF594E49FF5958121C3E563
:100C3C003394025002617F306502617FD802814E8D
:100C4C0061A8C26C53E67F759100855494855595C7
:100C5C00759104854E56854F57D26043E680D2AFCE
:0E0C6C00E52D54066008206A020533020C8A4A
:100C7A00306C0D206B0A2065071581158102150756
:100C8A002278003064053065027801E53775F0078F
:100C9A00A4F9E5F028F5F0E9A2F013A2F113A2F203
:100CAA0013F537C394785003753778C3E537953809
:100CBA004008D266D295D293D29730600281C48519
:100CCA005056855157D26043E68022207D11C2AF2B
:100CDA00754302C296D294D2AF759F11020EA4C276
:100CEA00AF754302C296D292D2AF759F11020EA47B
:100CFA00307243207D20C2AF754303900141757E57
:100D0A0040D293C292306204C297A118D296D2AF4F
:100D1A00759F13020EA4C2AF754303900141757EFD
:100D2A0040D295C294306204C297A138D296D2AF0B
:100D3A00759F10020EA4207D17C2AF754303900160
:100D4A001CD293306202C297D2AF759F13020EA4CF
:100D5A00C2AF75430390011CD295306202C297D28A
:100D6A00AF759F10020EA4207D11C2AF754304C255
:100D7A0094D292D2AF759F10020EA4C2AF754304EB
:100D8A00C292D294D2AF759F13020EA4307243203E
:100D9A007D20C2AF754305900130757E10D297C28F
:100DAA0096306204C295A1B4D294D2AF759F110253
:100DBA000EA4C2AF754305900152757E04D297C244
:100DCA0096306204C293A1D4D292D2AF759F110217
:100DDA000EA4207D17C2AF754305900112D2973039
:100DEA006202C295D2AF759F11020EA4C2AF7543BB
:100DFA0005900126D2973062EBC293D2AF759F114C
:100E0A00020EA4207D11C2AF754306C292D296D2B9
:100E1A00AF759F13020EA4C2AF754306C294D29651
:100E2A00D2AF759F10020EA4307242207D20C2AF4D
:100E3A00754301900152757E04D295C294306204C2
:100E4A00C293C150D292D2AF759F10020EA4C2AF04
:100E5A00754301900130757E10D293C292306204BC
:100E6A00C295C170D294D2AF759F13C1A4207D16CA
:100E7A00C2AF754301900126D295306202C293D265
:100E8A00AF759F10C1A4C2AF754301900112D293EE
:100E9A00306202C295D2AF759F13C26622900110CA
:100EAA00757E00D295D293D297C294C292C296C24C
:100EBA006222788076FF0876FF0876FF0876FF08B8
:100ECA00760308760408760A087603087601087617
:100EDA0001788C76010876FF0876FF0876FF087697
:100EEA00FF0876FF0876030876FF0876FF0876FF84
:100EFA000876250876D00876FA0876FA087604087D
:100F0A0076FF08760108760008767A0876FF087672
:100F1A0001087601087600087603227887E6FFC280
:100F2A0072BF0302D2727888E6C394036008C27D56
:100F3A00E630E102D27DC27E7889E630E102D27ED5
:100F4A00C3EF94026008758E01D273020F5D758E2D
:100F5A0000C273227880E6149000809378A4F67811
:100F6A0081E6149000809378A5F67886E6149000BE
:100F7A008D9378A6F6789CE67538FF75390CB4021D
:100F8A00067538A075390AB40306753882753905AD
:100F9A0078A3E61490009A93F569D1A7222278964D
:100FAA00E6FA7897E6FB7888E6B40305C3EB940E75
:100FBA00FB307F047A007BFFC3EB9AFCC394825018
:100FCA00027C827575000575EC8575F0A4C3E5F0A1
:100FDA00947D40F222D27FF1A812059C7A007B0010
:100FEA007C10120592E55F2AFA74003BFBDCF37C65
:100FFA0004C3EB13FBEA13FADCF7FEC27F120FA855
:10100A0022E5EF20E6037520000520903FFFE5204A
:10101A00146006901DFF1460009304600375EF12BC
:10102A0053D9BF7581C043FF8012058D75EF024306
:10103A00B203E5B3240420E70DF521E5E320E00639
:10104A008521B343E301120EA77580FF75A40075CD
:10105A00F1B275D4DF7590A975A5FC75F2FE75D548
:0F106A000175A60175E241E4F8F6D8FD756B013A
:10107900120EBC12154978988676753001C2AF12E6
:1010890005A61205B612059C1205BD12059C12058E
:10109900C412059C1216621205A61205A61205A114
:1010A900C2AF78FA79FA308507D9FBD8F7021C0064
:1010B900120F25120F5E120FA7120FA878988676C5
:1010C900120EA775885075891275C8247591047513
:1010D900D84075A82275B80275E690759B80759DF4
:1010E9000075D10E75BC5875BB0875BA1175E880C5
:1010F90012058DD2AF12084653DACF207E0343DAA8
:1011090020307E0343DA1043DA01C2D8C2711205D6
:10111900A6D2617B037A0CE55E70077A0CDB0302C9
:1011290010A912059C2070030210A9C270E55FC3C3
:10113900940240E1E52F541F856160F561B560D5E2
:10114900DAD5C26153DACF207E0343DA20307E0339
:1011590043DA10C2D8C27178A2E67008D274E52FBA
:1011690054E0F52FC2757529001205A1307409C321
:10117900E529940A4002D275120592780230740268
:101189007800C3E55F9840F0C2AF1205B61205B604
:101199001205B6D2AF1205A6754D007888E6B403DC
:1011A900024189120592788CE6C394015003021218
:1011B90089E530C394015003021289207435C3E5CF
:1011C9005F94FF5003021289C2AF1205CBD2AF124E
:1011D90005A1C3E55F940150EFC2AF1205B6120530
:1011E900971205B6D2AF1205A1C3E55F94FF40E996
:1011F9000216E77F05D27F120FA81205A1C2AFC25E
:101209007F120FA8AE5FC3E55F947FD2AF407B1218
:10121900058DC2AF1205CBD2AFDFDA120FDFC3EEF5
:1012290094057897F61205A612158B12166A7F0A8D
:10123900D27F120FA81205A1C2AFC27F120FA8AEAA
:101249005FC3E55F947FD2AF50E412058DC2AF1240
:1012590005B61205971205B6D2AFDFD4120FDFEE2D
:1012690024057896F61205A612158B121699120501
:10127900A1120FA8C3E55F94FF500221C40216E72B
:10128900C3E55F954D4003855F4D1205A17801794E
:1012990088E7B403027805C3E55F98400221A4C238
:1012A900AF1205CB1205CB1205CBD2AF1205A6752D
:1012B9003000E4F531F5320531E531F470390532A4
:1012C900789AE67819146012783214600D787D14D2
:1012D900600878FA146003753200C3E53298401744
:1012E90015327531B478998676C2AF1205CBD2AF73
:1012F900789886761205A1120597E52A700530744B
:101309000201A978012074027806C3E55F9840A715
:101319007888E6C3940360031205A1E52A700302E5
:1013290010A9C2AF120EA7E4F522F523F524F5257D
:10133900F526F56AD2AF7885E6C333F568E4F54555
:10134900F546F547F548F549F573F52CF52DF537CB
:1013590075730875BB1012058D12084AE5E820EC73
:10136900FBA8BDA9BEE97001F8887412084E75730F
:101379000875BB107887E6FE7602120F257887EE8E
:10138900F6C2AF7564FF1208C68522648522658599
:101399002266D2AF752201752401752501752601D2
:1013A90085636C756D017888E6B40307C27D307674
:1013B90002D27DD268D269753300120E0D120E3237
:1013C9001208E61208ED1208E61208ED1208E60204
:1013D90013E8C2AF120F25D2AF75730075BB08129F
:1013E9000B71120696120C8B120CD51208ED120B0A
:1013F90060306D031206972067031207E93067030F
:10140900120830120C8B120CFA1208ED120B713003
:101419006D031206D3120C8B120D711208ED120B0B
:1014290060306D03120731120C8B120D961208ED04
:10143900120B71306D0312078E120C8B120E0D12E6
:1014490008ED12084A120B60120C8B120E321208A8
:101459004E1208ED306932206B2F85676485676508
:0E14690085636C756D0179187A0CC3E53399B3
:10147700400CC269D26A8A357564FF021492C3E5CB
:101487005F940140030213E802150F306A1B206BBB
:1014970018E535147004C26A61DBF535C3E55F945E
:1014A7000140030213E802150F753600C3E56278A1
:1014B70082985054307404E52A604D7888E6B40366
:1014C70017207D0520760781DF30760281DF206BCC
:1014D70007D26B856764812778F0306B0585676471
:1014E7007820C3E54198500261E8306B1BC26BC29C
:1014F7007D307602D27DD26A75351285676461E8E0
:101507000536E55F6002A112753600C2AF120EA75D
:101517007887E6FE7602120F257887EEF6E4F52245
:10152700F523F524F525F526F568C268D2AF12052F
:101537008D120EA7307409C3E5369405400201A940
:1015470041BB901A0D78201215CDE520B45A0CA393
:101557001215CDE520B4A50302156B120EBC1215AA
:101567008B02158A901A0378807B0A1215CDA3087F
:10157700DBF9901A0F788C7B181215CDA308DBF9CD
:10158700901A2722C2AF12160C1215E6901A007491
:101597000E1215D2A374041215D2A374141215D205
:1015A700901A0378807B0A1215D1A308DBF9901AE9
:1015B7000F788C7B181215D1A308DBF912161F12AE
:1015C70015FD901A2722E493F622E6438F01538FE5
:1015D700FD75EF0275B7A575B7F1F0538FFE22437E
:1015E7008F02438F0175EF0275B7A575B7F1901A92
:1015F7000DF0538FFC22901A0D745AB1D2901A0E27
:1016070074A5B1D2227A3079D07820901A40B1CD22
:10161700E520F709A3DAF7227A3079D0901A40E764
:10162700B1D209A3DAF922AB77A878BB0102798492
:10163700BB02027985BB03027986BB04027992BBA0
:1016470005027987BB060279A3BB0702799CBB0811
:10165700027988BB09027989E8F7227C051205A679
:10166700DCFB22C2AF1205B61205BD1205C4120576
:10167700CB1205971205B61205BD1205C41205CB8C
:101687001205971205B61205BD1205C41205CBD275
:10169700AF22C2AF1205CB1205C41205BD1205B6A3
:1016A7001205971205CB1205C41205BD1205B61215
:1016B70005971205CB1205C41205BD1205B6D2AFA8
:1016C70022AE77AF78C2AF1205B61205B61205B6CD
:1016D700120597DEF21205CB120597DFF8D2AF227B
:1016E700D16AD162D162757701757801757900D1B8
:1016F700C87C05AD5F1205A6C3ED955F70F5C3E520
:101707005F9401400AC3E55F94FF4032021723D17B
:101717002EB18BD16AC2AF75EF12D162DCD50579D4
:10172700C3E5799403500280C6D1620578E5771442
:1017370090009F93F808C3E57898500280AED16275
:10174700D1620577C3E577940A5002809C120EBCDC
:09175700B18BC2AF75EF12D16233
:0319FD0002100BCA
:101A00000E0414FFFFFFFF03040A0301015AA5019E
:101A1000FFFFFFFFFF03FFFFFF25D0FAFA04FF01DE
:081A2000007AFF01010003FF41
:101A4000235475726E6967794E6665743235412329
:101A500023424C48454C4923463333302320202031
:101A60002020202020202020202020202020202076
:101C0000C2AFC2D353D9BF7581C043B20343FF8073
:101C1000752438752503B1C975EF0275E24043F1AB
:101C20002053A4DF75D400D2857DFA780379E67C51
:101C300010752200752300901DD67B0675249875BB
:101C400025013085028142208508D8FBD9F9DCF7CF
:101C500081B4308508D8FBD9F9DCF781B4B189E4C7
:101C600093A3C39A6004DDC381B4DBDBB17B600264
:101C7000812B7B08E493FAA3B15CDBF87A30B15C8A
:101C8000752200752300B17BEAFCEBFDC3ED94FEE9
:101C9000400EB17B8A278B28ED30E0048A828B834B
:101CA000B17B7AC270D8C3ED94FE601350CEBD00F4
:101CB00025EC60097520007521FF0200008100A855
:101CC00027A9280809D804D90281D3B17FEA89AAB3
:101CD000F281C50D81A0C3ED94035049EDA2E092BD
:101CE000007AC5C3E5829400E583941C50902000DF
:101CF00010438F02438F0175B7A575B7F1F030001F
:101D00001FA827A9280809438F01538FFDD804D99C
:101D100002A12089AAE275B7A575B7F1F0A3A10DBC
:101D2000538FFC817C7AC1BD030CE493A3FAB140CC
:101D3000DCF8B138817C817EAA22AB23B15CEBFA5E
:101D4000EA6222752608C3E52313F523E52213F57D
:101D50002250066323A0632201D526EAB1C9B1C986
:101D600075260AEAF4200102D285300102C285B14B
:101D7000C9C3134002C201D526EB22B17FEAFB2082
:101D80008502A17F308502A184752608AE24AF2587
:101D9000C3EF13FFEE13FEB1CDB1C9C3EA13308513
:101DA000024480FA30E703632201C3E52313F523DD
:101DB000E52213F52250066323A0632201D526D91C
:101DC000E52265236523F52222AE24AF250E0FDE22
:101DD000FEDFFCD20122424C48656C693437316326
:041DE000F3300601D5
:00000001FF
